:100000000C9479010C94A1010C94A1010C94A10110
:100010000C94A1010C94A1010C94A1010C94A101D8
:100020000C94A1010C94A1010C94A1010C94A101C8
:100030000C94A1010C94A1010C94A1010C94A101B8
:100040000C9432040C94A1010C94FA020C94D40286
:100050000C94A1010C94A1010C94A1010C94A10198
:100060000C94A1010C94A101467265652052414D8A
:100070003A20004552524F523A200053797320766D
:100080006F6C74733A200053797320766F6C7473BD
:10009000206368617267696E673A20005379732044
:1000A000766F6C74732069646C653A2000626174C9
:1000B00074506C757350696E204F4E006261747499
:1000C000506C757350696E204F46460063757272AE
:1000D000656E745A65726F4F66667365743A005345
:1000E000616D706C652073697A653A20003E00206E
:1000F0000020002000200020002000200020002000
:10010000003C0041444A555354494E472000616425
:100110006A416D70735F4F4E200061646A566F6C68
:1001200074735F4F4E200063656C6C5368756E741A
:10013000335F4F4E200063656C6C5368756E74328C
:100140005F4F4E200063656C6C5368756E74315F51
:100150004F4E200074617267657420416D70733A70
:10016000200074617267657420566F6C74733A2056
:100170000070777250574D3A200049444C45205446
:100180004F54414C20566F6C74733A200049444CD4
:100190004520566F6C747320333A200049444C4517
:1001A00020566F6C747320323A200049444C45202D
:1001B000566F6C747320313A2000434841524749CE
:1001C0004E4720544F54414C20566F6C74733A2064
:1001D000004348415247494E4720566F6C74732084
:1001E000333A20004348415247494E4720566F6CEE
:1001F000747320323A20004348415247494E472009
:10020000566F6C747320313A20004348415247497D
:100210004E472063757272656E7420414D50533A9B
:100220002000544F54414C20766F6C74733A200078
:10023000766F6C747320333A2000766F6C74732081
:10024000323A2000766F6C747320313A2000437587
:100250007272656E7420416D70733A200000000068
:1002600000240027002A0000000000250028002BA1
:10027000000404040404040404020202020202034F
:100280000303030303010204081020408001020459
:100290000810200102040810203C76657273696F13
:1002A0006E20302E3935373E003E003C7361666566
:1002B00043757272656E743A20003E003C7361664D
:1002C0006543757272656E743A20003E003C646F3F
:1002D000636B566F6C746167653A2000000000081C
:1002E00000020100000304070000000000000000FD
:1002F000102611241FBECFEFD8E0DEBFCDBF15E022
:10030000A0E0B1E0E2E3F2E502C005900D92A83072
:10031000B107D9F726E0A8E0B5E001C01D92A139E8
:10032000B207E1F711E0C9E7D1E004C02197FE016F
:100330000E940C29C837D107C9F70E9482100C947B
:1003400017290C940000CF92DF92EF92FF920F9347
:100350001F93CF93DF936C017A018B01C0E0D0E053
:10036000CE15DF0589F0D8016D918D01D601ED9193
:10037000FC910190F081E02DC6010995892B11F4C3
:100380007E0102C02196ECCFC701DF91CF911F9172
:100390000F91FF90EF90DF90CF900895089580E047
:1003A00090E00895FC01538D448D252F30E0842F7B
:1003B00090E0821B930B541710F0CF96089501978D
:1003C0000895FC01918D828D981761F0828DDF0177
:1003D000A80FB11D5D968C91928D9F5F9F73928F38
:1003E00090E008958FEF9FEF0895FC01918D828D2D
:1003F000981731F0828DE80FF11D858D90E00895FA
:100400008FEF9FEF0895FC01918D228D892F90E051
:10041000805C9F4F821B91098F739927089588EE06
:1004200095E00E94030221E0892B09F420E0822F4D
:100430000895FC01848DDF01A80FB11DA35ABF4FA1
:100440002C91848D90E001968F739927848FA689D3
:10045000B7892C93A089B1898C9180648C93938DFA
:10046000848D981306C00288F389E02D80818F7DEA
:1004700080830895EF92FF920F931F93CF93DF93A2
:10048000EC0181E0888F9B8D8C8D981305C0E889E5
:10049000F989808185FD24C0F62E0B8D10E00F5F59
:1004A0001F4F0F731127E02E8C8DE8120CC00FB672
:1004B00007FCFACFE889F989808185FFF5CFCE0165
:1004C0000E941902F1CF8B8DFE01E80FF11DE35A56
:1004D000FF4FF0820B8FEA89FB898081806207C021
:1004E000EE89FF896083E889F9898081806480834F
:1004F00081E090E0DF91CF911F910F91FF90EF90FD
:100500000895CF93DF93EC01888D8823C9F0EA89A1
:10051000FB89808185FD05C0A889B9898C9186FDFC
:100520000FC00FB607FCF5CF808185FFF2CFA889F9
:10053000B9898C9185FFEDCFCE010E941902E7CFDA
:10054000DF91CF91089580E090E0892B29F00E94FF
:100550000F0281110C94000008953FB7F894809128
:10056000E4059091E505A091E605B091E70526B573
:10057000A89B05C02F3F19F00196A11DB11D3FBFDB
:10058000BA2FA92F982F8827820F911DA11DB11D69
:10059000BC01CD0142E0660F771F881F991F4A9565
:1005A000D1F708950E9412291F920F920FB60F9251
:1005B00011242F933F934F935F936F937F938F9368
:1005C0009F93AF93BF93EF93FF9388EE95E00E94C4
:1005D0001902FF91EF91BF91AF919F918F917F9100
:1005E0006F915F914F913F912F910F900FBE0F90A0
:1005F0001F9018951F920F920FB60F9211242F93F0
:100600008F939F93EF93FF93E091F805F091F90595
:100610008081E091FE05F091FF0582FD12C090817E
:10062000809101068F5F8F7320910206821751F02F
:10063000E0910106F0E0E851FA4F958F80930106B2
:1006400001C08081FF91EF919F918F912F910F9029
:100650000FBE0F901F90189590E0FC01E452FD4FE3
:100660003491FC01EB57FD4F2491FC01EF58FD4FF5
:10067000E491EE2309F43BC0332339F1333091F098
:1006800038F43130A9F0323001F584B58F7D12C0D5
:10069000373091F03830A1F03430B9F480918000D7
:1006A0008F7D03C0809180008F77809380000DC084
:1006B00084B58F7784BD09C08091B0008F7703C067
:1006C0008091B0008F7D8093B000F0E0EE0FFF1FAF
:1006D000E959FD4FA591B4918FB7F894EC91611150
:1006E00003C020952E2301C02E2B2C938FBF08957D
:1006F000109264051092630580E090E00E94940ED1
:1007000010926105109262051092440585E090E018
:1007100090930B0180930A0160E088E00E942C0313
:100720001092670561E087E00E942C031092660535
:1007300061E084E00E942C03109265050895CF9338
:10074000DF9390E0FC01EB57FD4F2491FC01EF5843
:10075000FD4F8491882361F190E0880F991FFC017F
:10076000E35AFD4FC591D491FC01E959FD4FA59184
:10077000B491611109C09FB7F894888120958223B4
:100780008883EC912E230BC0623061F49FB7F894FC
:100790003881822F809583238883EC912E2B2C9394
:1007A0009FBF06C08FB7F894E8812E2B28838FBF98
:1007B000DF91CF9108958E3008F08E508770209190
:1007C000000190E4299F90011124822B80937C00EA
:1007D00080917A00806480937A0080917A0086FD0F
:1007E000FCCF809178002091790090E0922B0895C1
:1007F0008F929F92AF92BF92CF92DF92EF92FF9231
:100800006B017C010E94AD024B015C01C114D1045B
:10081000E104F104F1F00E94AD02DC01CB01881982
:100820009909AA09BB09883E9340A105B10570F357
:1008300021E0C21AD108E108F10888EE880E83E0B1
:10084000981EA11CB11CC114D104E104F10419F7D4
:10085000DDCFFF90EF90DF90CF90BF90AF909F9053
:100860008F9008951F920F920FB60F9211242F931D
:100870003F938F939F93AF93BF938091080590917F
:100880000905A0910A05B0910B053091E30523E01D
:10089000230F2D3720F40196A11DB11D05C026E8B8
:1008A000230F0296A11DB11D2093E3058093080537
:1008B00090930905A0930A05B0930B058091E40578
:1008C0009091E505A091E605B091E7050196A11D7F
:1008D000B11D8093E4059093E505A093E605B093E0
:1008E000E705BF91AF919F918F913F912F910F900D
:1008F0000FBE0F901F9018950C94712681309105B2
:1009000019F11CF4892B41F0089582309105A9F169
:10091000039709F484C00895809145059091460598
:10092000892B09F4EFC08091280590912905892B26
:1009300009F0E8C010924605109245051092E205B4
:100940001092E10560E0DBC020914505309146053D
:100950002130310509F4D6C02091280530912905B0
:10096000232B09F0CFC090934605809345059093C3
:10097000E2058093E10561E0C2C08091DD059091C0
:10098000DE05A091DF05B091E0050097A105B10556
:1009900039F020914505309146052230310571F03E
:1009A00082E090E0909346058093450581E090E0D9
:1009B0009093E2058093E10561E021C040916805D4
:1009C0005091690560916A0570916B054817590748
:1009D0006A077B0708F496C08091E1059091E205D3
:1009E000019729F41092E2051092E10506C081E01A
:1009F00090E09093E2058093E1056091E1058DE040
:100A00000E942C038091680590916905A0916A0568
:100A1000B0916B05845D9E4FAF4FBF4F36C0809144
:100A2000280590912905892B09F06CC04091DD05BE
:100A30005091DE056091DF057091E005411551058B
:100A40006105710531F08091450590914605039748
:100A500029F183E090E0909346058093450581E07D
:100A600090E09093E2058093E10561E08DE00E94C3
:100A70002C038091680590916905A0916A05B09159
:100A80006B058A5B9F4FAF4FBF4F8093DD059093FF
:100A9000DE05A093DF05B093E00508958091680519
:100AA00090916905A0916A05B0916B05841795072F
:100AB000A607B70738F12091E1053091E205213012
:100AC000310549F41092E2051092E10584529A4FE3
:100AD000AF4FBF4F0AC021E030E03093E2052093D2
:100AE000E1058A5B9F4FAF4FBF4F8093DD05909329
:100AF000DE05A093DF05B093E0056091E1058DE090
:100B00000C942C03089561E082E00E942C03109263
:100B1000220180915705882321F087E892E00C9408
:100B2000860E089560E082E00E942C0380912201ED
:100B3000811108C080915705882321F08FE992E048
:100B40000E94860E81E08093220108950F931F93E7
:100B5000CF938C010E946926C82FC80101960E947C
:100B600069262C2F30E0A901582BCA01CF911F9183
:100B70000F910895FF920F931F93CF93DF9389EB0B
:100B800092E00E942D108091010190910201449702
:100B900021F0C4E1D0E0F12C17C087EC92E034C022
:100BA000CE010E94A6058C01FF2021F08AEC92E084
:100BB0000E942D10B801012E000C880B990B0E9489
:100BC00003102296FF24F394209101013091020139
:100BD00021503109C217D3071CF380912805909149
:100BE00029050817190771F08AEC92E00E942D1070
:100BF0006091280570912905072E000C880B990B30
:100C00000E94031088EC92E0DF91CF911F910F9129
:100C1000FF900C94860E1F93CF93DF93192FEB0157
:100C2000682FCE010E947C04612FCE010196DF91D6
:100C3000CF911F910C947C040E9478031092600560
:100C400080E090E00C947E042F923F924F925F924E
:100C50006F927F928F929F92AF92BF92CF92DF92CC
:100C6000EF92FF920F931F93CF93DF93EC010797BF
:100C700011F4C0E0D0E083E3C82EDC2C83E7E82E3B
:100C800080E4F82E812C912C90E6A92E90E4B92EC8
:100C90002DEC422E2CEC522E2CE5622E20E4722EEE
:100CA00004E110E08091280590912905C817D90723
:100CB000C1F12097B1F12090010130900201C330C1
:100CC000D10551F424E12216310431F0C10102971B
:100CD0000E94A6050397F9F0B101CE010E940B0610
:100CE00060910101709102016E5F7F4F80E090E0A2
:100CF0000E940B068091010190910201029690934F
:100D000002018093010180915705882321F08CEC2A
:100D100092E00E94860ED0932905C09328050E9478
:100D2000BA05D0932905C093280582E090E00E947F
:100D30007E048091280590912905009719F087304D
:100D4000910529F480E090E00E947E045BC084312C
:100D500091050CF457C09C0124513109243131050F
:100D600098F50E941C0686E696E6A6E7B0E4809316
:100D7000390190933A01A0933B01B0933C01C0929A
:100D80008906D0928A06E0928B06F0928C068092B9
:100D90002B0190922C01A0922D01B0922E01409235
:100DA0002701509228016092290170922A0180E067
:100DB00090E0A0E0BFE38093230190932401A093EF
:100DC0002501B09326011EC09C012852310924310F
:100DD000310528F4109205010E941C0613C09C01E5
:100DE0002C5331092431310508F4BBCF80559109CA
:100DF000449740F4109205010E941C0684EE92E094
:100E00000E94860E8091010190910201843A9140E6
:100E1000E4F00E943807811118C01093020100937A
:100E2000010164E170E080912805909129050E94FC
:100E30000B068091010190910201029690930201AC
:100E400080930101CEE3D0E02DCFDF91CF911F91B0
:100E50000F91FF90EF90DF90CF90BF90AF909F9059
:100E60008F907F906F905F904F903F902F9008955C
:100E70000F931F93CF93DF93009101011091020113
:100E8000C4E1D0E00C171D073CF0CE010E94A6057E
:100E90008897F4F42296F6CFC4E1D0E08091010166
:100EA0009091020101968C179D0734F060E0CE010D
:100EB0000E947C042196F2CF84E190E0909302019D
:100EC0008093010180E090E00E94240681E001C04F
:100ED00080E0DF91CF911F910F91089560E083E052
:100EE0000E942C0380915705882321F087EF92E020
:100EF0000E94860E8091200190912101019751F06E
:100F000060E072EE84E090E00E94F8038DE390E0F0
:100F10000C94240608958F929F92AF92BF92CF9225
:100F2000DF92EF92FF9210924705109248051092BF
:100F3000490510924A05809122018823D9F08091B9
:100F400063059091640518161906A4F02091850692
:100F50003091860640918706509188066091180569
:100F60007091190580911A0590911B050E940E271A
:100F700087FF0CC081E090E0FF90EF90DF90CF9072
:100F8000BF90AF909F908F900C9424068090100596
:100F900090901105A0901205B0901305A501940141
:100FA00060911405709115058091160590911705B3
:100FB0000E94A1269B01AC0168E17AEF88E29BEBDD
:100FC0000E94A1266B017C016093100570931105AE
:100FD000809312059093130520E030E0A9010E9450
:100FE0006D2818165CF42DEC3CEC4CEC5EE3C7016C
:100FF000B6010E946D2818165CF028C02DEC3CEC60
:101000004CEC5EEBC701B6010E940E2787FF1EC0A5
:101010008091DA059091DB05833091058CF0809208
:10102000100590921105A0921205B092130581E56A
:1010300090E00E9424061092DB051092DA0552C05F
:1010400001969093DB058093DA054CC01092DB0586
:101050001092DA0580915705882301F18EE093E024
:101060000E94860E209110053091110540911205C5
:1010700050911305C501B4010E940E27882371F019
:101080008DE193E00E942D10609110057091110583
:1010900080911205909113050E94321020E030E0FB
:1010A0004AE754E460911005709111058091120592
:1010B000909113050E94722820E030E04AE754E442
:1010C0000E94A2260E948527DC01CB0164E070E02B
:1010D000FF90EF90DF90CF90BF90AF909F908F9058
:1010E0000C940B06FF90EF90DF90CF90BF90AF90E5
:1010F0009F908F9008958091DC0581111DC00E9402
:101100001C068FE293E00E94860E80916805909104
:101110006905A0916A05B0916B058053984FAF4F58
:10112000BF4F80933C0590933D05A0933E05B0933F
:101130003F0581E08093DC050895CF92DF92EF9226
:10114000FF92209120053091210540912205509178
:1011500023056091240570912505809126059091C5
:1011600027050E94A22620911C0530911D05409163
:101170001E0550911F050E94A2266B017C0120E0F4
:1011800030E040E450E460912B0170912C0180919B
:101190002D0190912E010E9472289B01AC01C70184
:1011A000B6010E940E2787FF18C02DEC3CEC44E8E6
:1011B00050E46091390170913A0180913B01909126
:1011C0003C010E940E27811108C08DE290E0FF9043
:1011D000EF90DF90CF900C9424060E941C062DEC1B
:1011E0003CEC44E850E46091390170913A018091FF
:1011F0003B0190913C010E940E27811118C0809103
:101200001C0190911D01A0911E01B0911F018093BE
:101210004B0590934C05A0934D05B0934E058AE382
:1012200093E0FF90EF90DF90CF900C94860EFF90AC
:10123000EF90DF90CF900895CF92DF92EF92FF92E0
:1012400020912805309129052330310559F16B0192
:101250007C0181E0809360050E947803809168059D
:1012600090916905A0916A05B0916B058C0D9D1D4B
:10127000AE1DBF1D6C017D0124ECC20E29E0D21E03
:10128000E11CF11CC0925305D0925405E092550523
:10129000F092560580930C0590930D05A0930E05D2
:1012A000B0930F05FF90EF90DF90CF90089580915D
:1012B0006305909164050E94940E80916805909159
:1012C0006905A0916A05B0916B05AC01BD014E5C4A
:1012D0005F4F6F4F7F4F40934005509341056093A0
:1012E00042057093430540ED57E060E070E04093A5
:1012F000310150933201609333017093340188536C
:101300009F4FAF4FBF4F80935C0590935D05A093B7
:101310005E05B0935F05109244050895AF92BF92A9
:10132000CF92DF92EF92FF920F931F93CF93DF93B1
:10133000C0912A05D0912B05C133D10509F58AEF5B
:1013400094E00E94860E80916705882359F084E41A
:1013500093E00E94860E60E088E00E942C031092C9
:1013600067050BC08FE493E00E94860E61E088E081
:101370000E942C0381E0809367058AEF94E04FC2BE
:10138000C233D105F9F48AEF94E00E94860E809171
:101390006605882359F089E593E00E94860E61E096
:1013A00087E00E942C031092660575C184E693E0E5
:1013B0000E94860E60E087E00E942C0381E080930B
:1013C000660569C1C333D105F9F48AEF94E00E9440
:1013D000860E80916505882359F08EE693E00E9481
:1013E000860E61E084E00E942C031092650553C1D3
:1013F00089E793E00E94860E60E084E00E942C035F
:1014000081E08093650547C1C033D105F9F460E000
:1014100088E00E942C0361E087E00E942C0361E0D9
:1014200084E00E942C038AEF94E00E94860E83E8F9
:1014300093E00E94860E8AEF94E00E94860E10923E
:101440006705109266051092650589C1C136D10500
:10145000B9F480E090E00E94940E8AEF94E00E943C
:10146000860E82E993E00E94860E8AEF94E00E9445
:10147000860E109264051092630580E090E04DC1E5
:10148000C236D10599F484E690E00E94940E8AEF6A
:1014900094E00E94860E8EE993E00E94860E8AEF09
:1014A00094E00E94860E84E690E02BC0C336D105FE
:1014B00099F488EC90E00E94940E8AEF94E00E94E8
:1014C000860E8CEA93E00E94860E8AEF94E00E94DA
:1014D000860E88EC90E015C0C436D105B9F48FEFC4
:1014E00090E00E94940E8AEF94E00E94860E8AEBB0
:1014F00093E00E94860E8AEF94E00E94860E8FEFA2
:1015000090E0909364058093630507C1C536D105CB
:10151000C9F48AEF94E00E94860E809162058823C8
:1015200039F01092620588EC93E00E942D10B3C050
:1015300081E08093620585ED93E00E942D100E946A
:101540005709A9C0C636D10529F58AEF94E00E9453
:10155000860E80916105882339F01092610581EE35
:1015600093E00E942D1009C081E0809361058DEE0B
:1015700093E00E942D100E9457098AEF94E00E9488
:10158000860E109258051092590510925A05109225
:101590005B05E5C0C937D105E9F42DEC3CEC4CE422
:1015A0005DE3609114017091150180911601909195
:1015B00017010E94A2266093140170931501809375
:1015C0001601909317018AEF94E00E94860E88EF2F
:1015D00093E05FC0C836D105E9F42DEC3CEC4CE457
:1015E0005DE3609114017091150180911601909155
:1015F00017010E94A1266093140170931501809336
:101600001601909317018AEF94E00E94860E8AE0FB
:1016100094E03FC0C537D105E9F42AE037ED43EA4D
:101620005CE3609110017091110180911201909121
:1016300013010E94A2266093100170931101809300
:101640001201909313018AEF94E00E94860E8CE1C0
:1016500094E01FC0CA36D10519F52AE037ED43EAF8
:101660005CE36091100170911101809112019091E1
:1016700013010E94A12660931001709311018093C1
:101680001201909313018AEF94E00E94860E8FE27C
:1016900094E00E94860E8AEF94E00E94860E5FC05E
:1016A000C936D105E1F48AEF94E00E94860E84E405
:1016B00094E00E94860E8AEF94E00E94860E80914C
:1016C0006305909164050A968F3F910519F014F017
:1016D0008FEF90E090936405809363051AC0CB363A
:1016E000D105F1F48AEF94E00E94860E8FE494E035
:1016F0000E94860E8AEF94E00E94860E8091630518
:10170000909164050A9797FFE5CF109264051092B7
:10171000630580916305909164050E94940E1FC03B
:10172000CF36D105E1F48AEF94E00E94860E8AE577
:1017300094E00E94860E8AEF94E00E94860E8091CB
:1017400063059091640501968F3F910519F014F09F
:101750008FEF90E090936405809363051AC0CC36B8
:10176000D10539F58AEF94E00E94860E84E694E074
:101770000E94860E8AEF94E00E94860E8091630597
:1017800090916405019797FFE5CF10926405109240
:1017900063058091630590916405DF91CF911F915E
:1017A0000F91FF90EF90DF90CF90BF90AF900C948F
:1017B000940EC736D105C9F48AEF94E00E94860ED4
:1017C00080916005882339F08AE991E00E94860EB5
:1017D0000E941C06D2CD80E891E00E94860E60E057
:1017E00070E0CB010E941C09C8CDCA37D10561F455
:1017F000DF91CF911F910F91FF90EF90DF90CF90ED
:10180000BF90AF900C948B07C637D105D1F480916F
:101810000501882381F0109205018EE694E0DF91A6
:10182000CF911F910F91FF90EF90DF90CF90BF90DD
:10183000AF900C94860E81E0809305018BE794E0D5
:10184000EECFC837D10519F487E894E0E8CFC13767
:10185000D10559F480915705882319F01092570546
:101860002DC281E08093570529C2C237D10561F4AA
:10187000DF91CF911F910F91FF90EF90DF90CF906C
:10188000BF90AF900C946E07C437D10561F461E04E
:1018900083E00E942C0380915705882309F40EC22F
:1018A00089E994E0BCCFCD36D10561F4DF91CF91C9
:1018B0001F910F91FF90EF90DF90CF90BF90AF906E
:1018C0000C949205CE36D10561F4DF91CF911F9132
:1018D0000F91FF90EF90DF90CF90BF90AF900C945E
:1018E0008305C037D10561F4DF91CF911F910F912E
:1018F000FF90EF90DF90CF90BF90AF900C947B085B
:10190000C737D105A9F48091680590916905A09128
:101910006A05B0916B05805A9541AF4FBF4F8093D8
:101920003C0590933D05A0933E05B0933F05C6C18D
:10193000C337D10519F1C433D105D9F480E090E063
:101940000E942406C4E1D0E080910101909102013F
:1019500001968C179D0734F060E0CE010E947C0454
:101960002196F2CF84E190E09093020180930101EF
:1019700005C0C234D10571F40E943807DF91CF91C0
:101980001F910F91FF90EF90DF90CF90BF90AF909D
:101990000C94BA05C334D105F1F4809128059091D7
:1019A00029050197879750F78091010190910201D5
:1019B000449721F380E090E00E9424068091010189
:1019C000909102010297909302018093010160E0DF
:1019D0000E947C04D3CFC533D105D1F480912E056C
:1019E000B82EA12C80912C05A82AB50180E090E0AA
:1019F0000E94BB2760931C0170931D0180931E0100
:101A000090931F0162E070E0C5010E940B0603C0C5
:101A1000C633D10569F48FEA94E00E942D106091DD
:101A20001C0170911D0180911E0190911F01DAC06F
:101A3000C634D10579F560912C0570912D05072EDE
:101A4000000C880B990B0E94BD2720911C0130913E
:101A50001D0140911E0150911F010E94722820E03B
:101A600030E048EC52E40E94132760934B057093DA
:101A70004C0580934D0590934E058EEB94E00E94AB
:101A80002D1060914B0570914C0580914D05909102
:101A90004E05A8C0C733D10519F489E992E002C107
:101AA000C833D10571F4C0E0D0E060E0CE010E94FF
:101AB0007C042196C11582E0D807B9F785EC94E043
:101AC000AECEC933D105D9F490912C0520913A05B9
:101AD00030913B052330310519F480912E0501C06A
:101AE00080E0D82EC12CC92AC6010E94240684E0B9
:101AF000C816D10409F0E2C08BEC91E090CEC1345D
:101B0000D10519F560914B0570914C0580914D05FB
:101B100090914E050E948527DC01CB0160E070E0CA
:101B20000E940B068091680590916905A0916A0555
:101B3000B0916B0580934F0590935005A09351058C
:101B4000B093520585ED94E06ACEC434D10509F016
:101B50004EC080912E05F82EE12C80912C05E701D6
:101B6000C82BBE010D2E000C880B990B0E94BD27BF
:101B700020E030E04AE754E40E9413276B017C0127
:101B800024E333E347E451E40E946D2818160CF077
:101B900095C0C0923501D0923601E0923701F092A3
:101BA00038012AE939E949E15FE3C701B6010E943A
:101BB000A12660938506709386068093870690938E
:101BC000880666E070E0CE010E940B0689EE94E084
:101BD0000E942D106091350170913601809137017E
:101BE000909138010E942F1088EC92E018CEC534F5
:101BF000D10589F48DEC92E00E945310609135017B
:101C00007091360180913701909138010E942F1018
:101C10008BEC92E047C0C734D10589F48CEB92E09D
:101C20000E94531060910601709107018091080194
:101C3000909109010E942F108AEB92E033C0C834C2
:101C4000D105E1F580912E05182F00E080912C053B
:101C5000082B68E070E0C8010E940B06B801110F64
:101C6000880B990B0E94BD2720E030E04AE754EC36
:101C70000E94132760930601709307018093080167
:101C8000909309018BEA92E00E9453106091060143
:101C90007091070180910801909109010E942F1015
:101CA00089EA92E0DF91CF911F910F91FF90EF9021
:101CB000DF90CF90BF90AF900C947410DF91CF91D4
:101CC0001F910F91FF90EF90DF90CF90BF90AF905A
:101CD0000895E091E805F091E9050190F081E02D8B
:101CE000682F88EE95E00994009769F0FC01019057
:101CF0000020E9F73197AF01481B590BBC0188EE72
:101D000095E00C94A30180E090E00895CF93DF93D9
:101D10000E94740EEC0188EF94E00E94740E8C0F08
:101D20009D1FDF91CF910895CF93DF93EC0161E088
:101D300085E00E949F03209711F460E004C0CF3F2C
:101D4000D10531F461E085E0DF91CF910C942C0353
:101D5000E1EEF2E0E491E330F9F048F4E130B9F07B
:101D6000E230A1F584B5806284BDC8BD34C0E730DF
:101D7000E9F0E83019F1E43049F5809180008062A3
:101D800080938000D0938B00C0938A0024C084B5D8
:101D9000806884BDC7BD1FC080918000806880932B
:101DA0008000D0938900C093880015C08091B00056
:101DB00080688093B000C093B3000DC08091B000E4
:101DC00080628093B000C093B40005C0C038D105D4
:101DD0000CF0B8CFB2CFDF91CF9108958F929F9240
:101DE000AF92BF920F931F93CF93DF93CDB7DEB720
:101DF000A1970FB6F894DEBF0FBECDBF19A2423037
:101E000008F44AE08E010F5D1F4F842E912CA12C07
:101E1000B12CA50194010E947F26E62FB901CA01C9
:101E200001501109EA3014F4E05D01C0E95CD80109
:101E3000EC93232B242B252B61F7C8010E94740EF1
:101E4000A1960FB6F894DEBF0FBECDBFDF91CF9144
:101E50001F910F91BF90AF909F908F9008954F92D8
:101E60005F926F927F928F929F92AF92BF92CF922A
:101E7000DF92EF92FF926B017C01B42E9B01AC01CB
:101E80000E94DF28882319F08BEF94E027C02601F9
:101E90003701E89477F82FEF3FEF4FE75FE7C30193
:101EA000B2010E94DF2881110DC02FEF3FEF4FE7F5
:101EB0005FE7C301B2010E940E2718161CF48FEFD2
:101EC00094E00CC02FEF3FEF4FE75FE4C701B6018E
:101ED0000E946D28181684F483E095E0FF90EF903F
:101EE000DF90CF90BF90AF909F908F907F906F903A
:101EF0005F904F900C94740E2FEF3FEF4FE75FEC25
:101F0000C701B6010E940E2787FDE6CF20E030E032
:101F1000A901C701B6010E940E2787FF09C08DE203
:101F20000E94690E4C01F7FAF094F7F8F09402C0A1
:101F3000812C912CA12C60E070E080E09FE3AB1439
:101F400041F020E030E040E251E40E941327A394E6
:101F5000F6CF9B01AC01C701B6010E94A2262B015E
:101F60003C010E948C276B017C010E94BB279B01D6
:101F7000AC01C301B2010E94A1262B013C014AE041
:101F8000C701B6010E94EE0E7C01E80CF91CBB20D3
:101F900029F08EE20E94690EE80EF91EDB2CDD208E
:101FA00021F120E030E040E251E4C301B2010E949F
:101FB00072282B013C010E948C274B01A12CB12CD3
:101FC0004AE0C501B4010E94EE0EE80EF91EC501FB
:101FD000B4010E94BB279B01AC01C301B2010E9466
:101FE000A1262B013C01DA94DACFC701FF90EF90D4
:101FF000DF90CF90BF90AF909F908F907F906F9029
:102000005F904F900895CF92DF92EF92FF92CF931F
:10201000DF9397FF19C06B017C018DE20E94690E6E
:10202000EC0166277727CB016C197D098E099F0982
:102030004AE00E94EE0E8C0F9D1FDF91CF91FF9022
:10204000EF90DF90CF9008954AE0DF91CF91FF901D
:10205000EF90DF90CF900C94EE0E0C94740E42E053
:102060000C942F0FCF93DF9342E00E942F0FEC01CF
:1020700088EF94E00E94740E8C0F9D1FDF91CF912A
:102080000895CF93DF93BC01990F880B990B0E94A1
:102090000310EC0188EF94E00E94740E8C0F9D1FDA
:1020A000DF91CF9108950F931F93CF93DF938C010E
:1020B000C0E0D0E0F801EC0FFD1F6491662371F0E1
:1020C000E091E805F091E9050190F081E02D88EEBE
:1020D00095E00995892B11F02196ECCFCE01DF9187
:1020E000CF911F910F910895CF93DF930E945310CA
:1020F000EC0188EF94E00E94740E8C0F9D1FDF911D
:10210000CF910895CF93DF93CDB7DEB72C970FB65D
:10211000F894DEBF0FBECDBF789484B5826084BDD5
:1021200084B5816084BD85B5826085BD85B58160DB
:1021300085BD80916E00816080936E001092810059
:102140008091810082608093810080918100816014
:1021500080938100809180008160809380008091D5
:10216000B10084608093B1008091B0008160809361
:10217000B00080917A00846080937A0080917A0028
:10218000826080937A0080917A00816080937A00E7
:1021900080917A00806880937A001092C10010923A
:1021A000000160E08EE00E949F0360E08FE00E94EB
:1021B0009F0360E080E10E949F0360E081E10E9454
:1021C0009F0360E082E10E949F0361E088E00E943B
:1021D0009F0361E087E00E949F0361E084E00E942A
:1021E0009F0360E088E00E942C0361E087E00E948A
:1021F0002C0361E084E00E942C0385B5887F816018
:1022000085BD61E08DE00E949F03609145058DE0F2
:102210000E942C0361E085E00E949F03809163058A
:10222000909164050E94940E61E083E00E949F03F8
:1022300061E083E00E942C0361E082E00E949F0342
:1022400060E082E00E942C03E091F805F091F9052E
:1022500082E08083E091F405F091F5051082E09131
:10226000F605F091F70580E1808310920006E09179
:10227000FC05F091FD0586E08083E091FA05F09180
:10228000FB05808180618083E091FA05F091FB0578
:10229000808188608083E091FA05F091FB05808160
:1022A00080688083E091FA05F091FB0580818F7D45
:1022B00080838FE491E00E94860E82E090E00E948D
:1022C000A6051816190674F4BC01990F880B990B12
:1022D0000E94BD2760931C0170931D0180931E0115
:1022E00090931F0180E090E00E94A605BC01990F29
:1022F000880B990B0E94BD276B017C0180901C010B
:1023000090901D01A0901E01B0901F01A5019401A5
:102310000E946D2818164CF480924B0590924C0543
:10232000A0924D05B0924E0508C0C0924B05D092C8
:102330004C05E0924D05F0924E0584E090E00E943D
:10234000A6050097B9F0BC01685E7340072E000C2B
:10235000880B990B0E94BD2720E030E04AE754E447
:102360000E94132760931005709311058093120546
:102370009093130586E090E00E94A605BC01990F9A
:10238000880B990B0E94BD2720E030E04AE754E417
:102390000E9413276B017C0124E333E347E451E4FB
:1023A0000E946D281816C4F4C0923501D0923601EF
:1023B000E0923701F09238012AE939E949E15FE317
:1023C000C701B6010E94A126609385067093860618
:1023D000809387069093880688E090E00E94A60587
:1023E000BC01895B9B40833C994058F5072E000C4B
:1023F000880B990B0E94BD2720E030E04AE754EC9F
:102400000E941327609306017093070180930801CF
:102410009093090116C00E94A6050097D1F09093F1
:102420002905809328058730910511F00E94240624
:102430008091010190910201029690930201809394
:1024400001018091010190910201893B31E09307E4
:1024500014F3AE014F5F5F4F5C834B832FB7F8944B
:10246000609108057091090580910A0590910B050E
:102470002FBF0E94BB2720E030E040E85CE30E94D1
:1024800072280E948C276B017C01809168059091D5
:102490006905A0916A05B0916B05C816D906EA06D0
:1024A000FB0640F4C092D605D092D705E092D8053D
:1024B000F092D905C0926805D0926905E0926A054C
:1024C000F0926B05E0916705E1111BC080916605F4
:1024D000811117C080916505811113C0809163053A
:1024E000909164051816190664F0809162058111B7
:1024F00008C080916105811104C080916005882326
:1025000021F081E08093D50502C01092D50580911D
:10251000310190913201A0913301B09134019701C2
:102520008601081B190B2A0B3B0B40915C0550914F
:102530005D0560915E0570915F0540175107620768
:10254000730708F075C0C816D906EA06FB0608F43A
:102550006FC02091D505222309F46AC0C0925C05A2
:10256000D0925D05E0925E05F0925F05803D974058
:10257000A105B105E9F480E090E00E94940E60E0CE
:1025800088E00E942C0361E087E00E942C0361E058
:1025900084E00E942C0388EC90E0A0E0B0E08093FF
:1025A000310190933201A0933301B09334012BC0D9
:1025B000EE2321F061E088E00E942C038091660503
:1025C000882321F060E087E00E942C03809165055C
:1025D000882321F060E084E00E942C038091630551
:1025E000909164050E94940E20ED37E040E050E0A9
:1025F00020933101309332014093330150933401E1
:1026000081E080936C0532E3C30ED11CE11CF11C08
:10261000C0924005D0924105E0924205F0924305F8
:10262000109258051092590510925A0510925B05A8
:10263000C0906805D0906905E0906A05F0906B0540
:102640008090580590905905A0905A05B0905B0570
:10265000D701C6018A5F9109A109B10988169906B7
:10266000AA06BB0608F0CEC64AEFC416D104E104A0
:10267000F10408F4C7C62090D3053090D405121495
:1026800013040CF0BFC68091C1059091C205B10141
:102690000E94E428072E000C880B990B0E94BD278E
:1026A0002FE632E143E850E40E94722820E030EC4B
:1026B0004FE754E40E94132720E030E040E250E46A
:1026C0000E94A12624EA30E74DE35EE30E9413272F
:1026D000209110053091110540911205509113057C
:1026E0000E94A2266D837E838F8398876093140552
:1026F0007093150580931605909317058114910426
:10270000A104B10409F442C0C701B60168197909EE
:102710008A099B090E94BB2720E03AEB4BE55AE46B
:102720000E9413272D813E814F8158850E94722877
:1027300020E030E04AE754E40E94722820914B05E3
:1027400030914C0540914D0550914E050E94A226B6
:1027500060934B0570934C0580934D0590934E0507
:10276000C0901C01D0901D01E0901E01F0901F014F
:10277000A70196010E946D28181644F4C0924B05DB
:10278000D0924C05E0924D05F0924E058091BF0528
:102790009091C005B1010E94E428072E000C880B1F
:1027A000990B0E94BD2720E030EC4FE754E40E94D3
:1027B00013272FE632E143E850E40E9472282AEF03
:1027C00039E146E55FE30E94132720E030E0A901EC
:1027D0000E94A2266B017C0160932405709325055D
:1027E00080932605909327058091BD059091BE05A5
:1027F000B1010E94E428072E000C880B990B0E945F
:10280000BD2720E030EC4FE754E40E9413272FE669
:1028100032E143E850E40E94722821EE3FE641EEA7
:102820005EE30E941327A70196010E94A12620E0E3
:1028300030E0A9010E94A2264B015C0160932005B3
:102840007093210580932205909323058091BB0509
:102850009091BC05B1010E94E4288B01A50194016F
:10286000C701B6010E94A22669877A878B879C8759
:10287000B801110F880B990B0E94BD2720E030ECA6
:102880004FE754E40E9413272FE632E143E850E477
:102890000E9472282FEF35EE42E95EE30E94132773
:1028A00029853A854B855C850E94A12620E030E091
:1028B000A9010E94A2262B013C0160931C05709384
:1028C0001D0580931E0590931F059B01AC01698532
:1028D0007A858B859C850E94A22669877A878B875B
:1028E0009C87209118013091190140911A01509153
:1028F0001B010E940E2787FF0CC089859A85AB8536
:10290000BC858093180190931901A0931A01B0938C
:102910001B018091B9059091BA05B1010E94E4288C
:10292000072E000C880B990B0E94BD2720E030EC8D
:102930004FE754E40E9413272FE632E143E850E4C6
:102940000E94722827E53FE348E65EE30E941327D2
:10295000609318057093190580931A0590931B05D1
:102960001092C2051092C1051092C0051092BF05C9
:102970001092BE051092BD051092BC051092BB05C9
:102980001092BA051092B905309284052092830501
:102990001092D4051092D3052091D505222309F475
:1029A000FFC020916C05222319F1C092A905D09295
:1029B000AA05E092AB05F092AC058092A505909235
:1029C000A605A092A705B092A8054092A105509235
:1029D000A2056092A3057092A40560939905709377
:1029E0009A0580939B0590939C0510926C05D8C026
:1029F000C092B505D092B605E092B705F092B80541
:102A00008092B1059092B205A092B305B092B40540
:102A10004092AD055092AE056092AF057092B00540
:102A200060939D0570939E0580939F059093A005EC
:102A30002D813E814F8158852093950530939605D1
:102A40004093970550939805A5019401C701B601DD
:102A50000E946D2887FD11C0A3019201C701B60134
:102A60000E946D2887FD09C0C0928B05D0928C050D
:102A7000E0928D05F0928E0521C0A7019601C50157
:102A8000B4010E946D2887FD11C0A3019201C50108
:102A9000B4010E946D2887FD09C080928B05909239
:102AA0008C05A0928D05B0928E0508C040928B05D2
:102AB00050928C0560928D0570928E052AE037ED5C
:102AC00043E25DE36091390170913A0180913B01ED
:102AD00090913C010E94A2269B01AC0160918B0564
:102AE00070918C0580918D0590918E050E946D28C6
:102AF0001816F4F4809160058823D1F08091630565
:102B000090916405059797FD05C0909364058093A7
:102B1000630504C010926405109263050E94570972
:102B200080915705882321F087E591E00E94860E69
:102B300020912301309124014091250150912601DB
:102B400060919505709196058091970590919805F3
:102B50000E94A12629E23CE54FE05EE30E946D2839
:102B60001816F4F4809160058823D1F080916305F4
:102B700090916405059797FD05C090936405809337
:102B8000630504C010926405109263050E94570902
:102B900080915705882321F08AE691E00E94860EF5
:102BA0008091680590916905A0916A05B0916B05C7
:102BB0008093580590935905A0935A05B0935B05EF
:102BC000C0901805D0901905E0901A05F0901B05EB
:102BD00020913501309136014091370150913801F3
:102BE000C701B6010E946D2887FD84C01092700550
:102BF00010926F058091200190912101019709F4B5
:102C0000DDC080916D0590916E05823091050CF4C8
:102C10006BC010926E0510926D0541E050E050932C
:102C200021014093200187E791E00E94860E809168
:102C30000501882309F4C2C0C0908906D0908A0695
:102C4000E0908B06F0908C06A70196016091240518
:102C50007091250580912605909127050E946D2889
:102C600087FD1FC0A7019601609120057091210585
:102C700080912205909123050E946D2887FD11C047
:102C8000A701960160911C0570911D0580911E059C
:102C900090911F050E946D2887FD03C00E949D082A
:102CA0008DC080915705882321F080E891E00E9433
:102CB000860E60E177E280E090E00E941C0980913E
:102CC000680590916905A0916A05B0916B058857D8
:102CD0009C4EAF4FBF4F8093470590934805A093FC
:102CE0004905B0934A056AC0019690936E0580939A
:102CF0006D0564C010926E0510926D05209120053F
:102D000030912105409122055091230560912405C1
:102D10007091250580912605909127050E94A22695
:102D200020911C0530911D0540911E0550911F05F5
:102D30000E94A2269B01AC01C701B6010E940E278A
:102D40001816C4F18091200190912101892BB1F1D5
:102D500080916F0590917005823091052CF1109251
:102D6000700510926F0510922101109220018FE8DA
:102D700091E00E94860E0E948305109247051092F2
:102D800048051092490510924A0580910501882353
:102D9000A9F080915705882321F08AE991E00E94EB
:102DA000860E0E941C060AC00196909370058093BF
:102DB0006F0504C01092700510926F0520912005D8
:102DC0003091210540912205509123056091240501
:102DD0007091250580912605909127050E94A226D5
:102DE00020911C0530911D0540911E0550911F0535
:102DF0000E94A2269B01AC016091180570911905F3
:102E000080911A0590911B050E946D28181614F5E3
:102E10008091030190910401019721F18091710546
:102E200090917205823091057CF01092720510929B
:102E3000710581E090E090930401809303018AEA98
:102E400091E00E94860E0EC00196909372058093C9
:102E5000710508C01092720510927105109204015C
:102E6000109203018091200190912101892B09F09A
:102E700079C1C0902701D0902801E0902901F090FD
:102E80002A01A70196016091240570912505809182
:102E90002605909127050E940E2787FD1CC0A701DB
:102EA00096016091200570912105809122059091F5
:102EB00023050E940E2787FD0EC0A7019601609191
:102EC0001C0570911D0580911E0590911F050E94A3
:102ED0000E2787FF31C0809175059091760580356A
:102EE000910524F110927605109275050E947B08D9
:102EF0002DEC3CEC4CE450E46091270170912801EA
:102F00008091290190912A010E940E27811118C0F9
:102F100086E090E00E94240680915705882309F4FA
:102F200021C186EB91E00E94860E1CC10196909310
:102F300076058093750504C010927605109275058C
:102F4000C0902405D0902505E0902605F090270537
:102F50002AE939E949E650E4C701B6010E940E2783
:102F600087FD20C02AE939E949E650E4609120054F
:102F70007091210580912205909123050E940E27D2
:102F800087FD10C02AE939E949E650E460911C0543
:102F900070911D0580911E0590911F050E940E27BE
:102FA00087FFDCC080917305909174058035910591
:102FB0000CF4CEC0109274051092730580914505F3
:102FC00090914605039709F4B6C0A70196016AE9F6
:102FD00079E989E690E40E94A12620E030E040E80B
:102FE0005EE30E940E2787FD2CC0209120053091C2
:102FF000210540912205509123056AE979E989E686
:1030000090E40E94A12620E030E040E85EE30E94C8
:103010000E2787FD16C020911C0530911D0540919B
:103020001E0550911F056AE979E989E690E40E943E
:10303000A12620E030E040E85EE30E940E2787FFF3
:103040007AC080901C0190901D01A0901E01B0904C
:103050001F0120914B0530914C0540914D05509139
:103060004E05C501B4010E94A12623E333E343E3E7
:103070005FE30E9413276B017C01A50194010E946C
:10308000A1262B013C0120E030E0A9010E946D281F
:10309000181624F077FA709477F87094A5019401CB
:1030A000C301B2010E9413272DEC3CEC4CE45EE31B
:1030B0000E946D281816BCF4A5019401C701B60141
:1030C0000E946D2818162CF42AE939E949E95FE3D2
:1030D00004C02DEC3CEC4CE45FE3C501B4010E945C
:1030E00072286B017C01C0921C01D0921D01E092FC
:1030F0001E01F0921F01C701B6010E948527DC0165
:10310000CB0162E070E00E940B062AE939E949E947
:103110005EE360911C0170911D0180911E019091F0
:103120001F010E94722860934B0570934C05809399
:103130004D0590934E0583E090E00E947E048091BF
:103140002F0190913001019769F40E947B080AC019
:103150000196909374058093730504C010927405D2
:103160001092730520912005309121054091220590
:1031700050912305609124057091250580912605C5
:10318000909127050E94A2262DEC3CEC4CE45EE3D6
:103190000E940E2787FF0BC083E090E00E94240668
:1031A00080910501882369F00E941C060AC0809165
:1031B000280590912905039721F480E090E00E9472
:1031C00024068091200190912101019729F010920D
:1031D0007805109277052FC02091850630918606DC
:1031E00040918706509188066091180570911905E5
:1031F00080911A0590911B050E940E2787FFE7CF4B
:103200008091770590917805843191057CF010923A
:103210007805109277058BEC91E00E94860E0E9453
:103220001C0684E090E00E94240605C0019690935D
:1032300078058093770526E636E646EE5EE36091F4
:1032400014057091150580911605909117050E943F
:103250006D281816D4F48091630590916405892B2C
:10326000A1F48091790590917A05853091053CF023
:1032700082E590E00E9424060E94920506C0019615
:1032800090937A058093790504C010927A05109284
:10329000790520E030E040E05FE360911405709133
:1032A000150580911605909117050E940E2787FF3E
:1032B00019C08091630590916405843B910591F458
:1032C00080917B0590917C05893291052CF08AE2F2
:1032D00090E00E94240606C0019690937C0580939E
:1032E0007B0504C010927C0510927B052091230180
:1032F00030912401409125015091260160911405DF
:103300007091150580911605909117050E94A126D0
:1033100029E23CE54FE05EE30E946D28181694F424
:1033200080917D0590917E05853191052CF083E596
:1033300090E00E94240606C0019690937E0580933B
:103340007D0504C010927E0510927D0520E030E0DE
:1033500040E05FE3609106017091070180910801F0
:10336000909109010E94A2269B01AC016091140575
:103370007091150580911605909117050E940E27F2
:1033800087FF15C08091810590918205833091055A
:103390004CF084ED91E00E94860E1092820510920E
:1033A000810505C001969093820580938105209147
:1033B0000601309107014091080150910901609187
:1033C00014057091150580911605909117050E94BE
:1033D0000E2787FF17C080917F059091800583306D
:1033E00091055CF082E090E00E9424060E946E0746
:1033F0001092800510927F0505C00196909380057C
:1034000080937F058091680590916905A0916A0578
:10341000B0916B058C019D01005D174021093109B8
:103420004091CF055091D0056091D1057091D205A2
:10343000401751076207730708F09CC2803D27E0E0
:103440009207A105B10508F495C240913101509150
:1034500032016091330170913401483C510561059E
:10346000710509F487C220915705222309F482C20D
:103470008093CF059093D005A093D105B093D2054A
:103480008091D505811157C08EE492E00E945310BF
:10349000609114057091150580911605909117059E
:1034A0000E94321084E492E00E945310609124053F
:1034B0007091250580912605909127050E94321074
:1034C0008AE392E00E9453106091200570912105DB
:1034D00080912205909123050E94321080E392E0B2
:1034E0000E94531060911C0570911D0580911E056E
:1034F00090911F050E94321082E292E00E945310C8
:1035000020912005309121054091220550912305FD
:1035100060912405709125058091260590912705DD
:103520000E94A22620911C0530911D0540911E0588
:1035300050911F05A2C08AE092E00E945310609152
:1035400095057091960580919705909198050E9438
:10355000321087EF91E00E9453106091B505709191
:10356000B6058091B7059091B8050E94321084EE9F
:1035700091E00E9453106091B1057091B205809165
:10358000B3059091B4050E94321081ED91E00E9444
:1035900053106091AD057091AE058091AF0590918B
:1035A000B0050E9432108AEB91E00E9453102091E6
:1035B000B1053091B2054091B3055091B4056091C9
:1035C000B5057091B6058091B7059091B8050E9438
:1035D000A2262091AD053091AE054091AF055091E6
:1035E000B0050E94A2260E9432108BEA91E00E9450
:1035F00053106091A9057091AA058091AB05909137
:10360000AC050E9432108CE991E00E945310609149
:10361000A5057091A6058091A7059091A8050E9427
:1036200032108DE891E00E9453106091A1057091D5
:10363000A2058091A3059091A4050E9432108AE70B
:1036400091E00E9453102091A5053091A60540916C
:10365000A7055091A8056091A9057091AA058091D0
:10366000AB059091AC050E94A2262091A105309156
:10367000A2054091A3055091A4050E94A2260E9494
:10368000321081E791E00E94531080916305909180
:1036900064050E94411082E691E00E9453106091FF
:1036A00010017091110180911201909113010E94FB
:1036B000321084E591E00E945310609114017091E2
:1036C000150180911601909117010E94321080918E
:1036D0006705882331F085E491E00E94531081E072
:1036E00001C080E090916605992329F086E391E07E
:1036F0000E94531081E090916505992329F087E29B
:1037000091E00E94531081E090916205992329F085
:103710008AE191E00E94531081E090916105992324
:1037200029F08EE091E00E94531081E090914405D1
:10373000992329F083E091E00E94531002C088236E
:1037400021F08AEF94E00E94860E81E091E00E94D1
:103750005310609168057091690580916A05909198
:103760006B054AE00E94EE0E8FEF90E00E9453102E
:103770008091D505882399F1609195057091960502
:1037800080919705909198050E942F108DEF90E001
:103790000E9453106091B5057091B6058091B705F0
:1037A0009091B8050E942F108BEF90E00E9453106B
:1037B0006091B1057091B2058091B3059091B40507
:1037C0000E942F1089EF90E00E9453106091AD0588
:1037D0007091AE058091AF059091B00532C06091B7
:1037E00014057091150580911605909117050E949A
:1037F0002F1087EF90E00E94531060912405709184
:10380000250580912605909127050E942F1085EFB0
:1038100090E00E94531060912005709121058091E5
:103820002205909123050E942F1083EF90E00E94C3
:10383000531060911C0570911D0580911E0590919B
:103840001F050E942F1081EF90E00E94531060919D
:1038500018057091190580911A0590911B050E9419
:103860002F108FEE90E00E945310609163057091CD
:103870006405072E000C880B990B0E9403108DEE37
:1038800090E00E9474108FED90E00E9453108091A0
:103890008305909184050E9441108CEC90E00E9479
:1038A000531060911005709111058091120590914F
:1038B00013050E94321080912201882319F08CEBAD
:1038C00090E002C08DEA90E00E9474108091D505CE
:1038D0008823D9F08CE990E00E94531060919905FB
:1038E00070919A0580919B0590919C050E943210E1
:1038F00087E890E00E94531060919D0570919E05AD
:1039000080919F059091A0050CC08BE790E00E94EC
:103910005310609118057091190580911A059091C6
:103920001B050E9432108091280590912905892B52
:1039300051F083E790E00E94531080912805909108
:1039400029050E94411088E690E00E945310809162
:103950008D0690918E06009711F481E996E04B81D7
:103960005C81481B590BCA010E9441108AEF94E008
:103970000E94860EC0906805D0906905E0906A05A7
:10398000F0906B05B701A6014A5F51096109710901
:103990008091CB059091CC05A091CD05B091CE053D
:1039A00084179507A607B70708F053C15AEFC51645
:1039B000D104E104F10408F44CC180916205811145
:1039C00005C090916105992309F443C1C092CB05CC
:1039D000D092CC05E092CD05F092CE058823C9F0B7
:1039E0008090100190901101A0901201B0901301ED
:1039F00080918B0590918C05A0918D05B0918E05DD
:103A00008D839E83AF83B8872AE037ED43EA5CE37A
:103A100018C08090140190901501A0901601B090EC
:103A200017018091950590919605A0919705B09109
:103A300098058D839E83AF83B88729E23CE54FE8E4
:103A40005DE329873A874B875C87A50194016D81E7
:103A50007E818F8198850E94A1262B013C0120E068
:103A600030E0A9010E946D28181624F077FA7094AE
:103A700077F8709429853A854B855C85C301B2013E
:103A80000E946D2887FDE3C0809144052090630566
:103A90003090640581114DC081E080934405C0924F
:103AA000D605D092D705E092D805F092D905A501A8
:103AB00094016D817E818F8198850E940E2787FFFA
:103AC00007C041E050E0509386054093850506C04D
:103AD0008FEF9FEF909386058093850520E030E07F
:103AE00040E850E469857A858B859C850E94722820
:103AF0009B01AC01C301B2010E946D2818161CF491
:103B000085E090E002C081E090E090930B0180930B
:103B10000A0140910A0150910B01209185053091D5
:103B20008605429FC001439F900D529F900D112426
:103B300046C0A50194016D817E818F8198850E9488
:103B40000E27009185051091860587FF12C00F3F53
:103B50009FEF190771F4A1E0B0E0B0930B01A093BF
:103B60000A01B0938605A0938505BFEF2B1A3B0A87
:103B700028C0A50194016D817E818F8198850E9466
:103B80006D2818168CF40130110571F410930B0197
:103B900000930A018FEF9FEF909386058093850530
:103BA00021E0221A31080DC020910A0130910B0149
:103BB000209FC001219F900D309F900D1124280E51
:103BC000391E3092640520926305809163059091BF
:103BD0006405853B91053CF084EB90E0909364058F
:103BE0008093630506C097FF04C01092640510928D
:103BF000630580916305909164050E94940ED7013E
:103C0000C601C296A11DB11D809340059093410548
:103C1000A0934205B093430580ED97E0A0E0B0E0AB
:103C20008093310190933201A0933301B09334011A
:103C3000D701C60188539F4FAF4FBF4F80935C059C
:103C400090935D05A0935E05B0935F0502C010924E
:103C50004405C0906805D0906905E0906A05F09031
:103C60006B05B701A601445C594061097109809157
:103C7000530590915405A0915505B09156058417B0
:103C80009507A607B70708F03CC394ECC91699E05E
:103C9000D906E104F10408F434C380916005882357
:103CA00009F42FC3C0925305D0925405E0925505F4
:103CB000F092560580910C0590910D05A0910E058E
:103CC000B0910F05A7019601281B390B4A0B5B0B1E
:103CD000DA01C90181309749A944B14068F0809167
:103CE0005705882321F083EE91E00E94860E0E9402
:103CF0001C068EE290E0E0C0809128059091290595
:103D0000039719F40E941C06FCC28090A9059090AC
:103D1000AA05A090AB05B090AC0524EA30E745E8D1
:103D200050E4C501B4010E946D28181604F124EA7C
:103D300030E745E850E46091A5057091A6058091B3
:103D4000A7059091A8050E946D28181684F024EA12
:103D500030E745E850E46091A1057091A20580919B
:103D6000A3059091A4050E946D281816B4F48091C3
:103D70009305909194058330910549F48BE290E08E
:103D80000E9424061092940510929305BAC20196DF
:103D9000909394058093930504C01092940510921B
:103DA00093052DEC3CEC4CE45EE36091950570913D
:103DB000960580919705909198050E940E2787FFA0
:103DC0001AC0809162058823B1F080918F0590918F
:103DD0009005A0919105B0919205C81AD90AEA0AF6
:103DE000FB0A41E6C4164AEED406E104F10458F099
:103DF0000E949D0886C2C0928F05D0929005E092E5
:103E00009105F092920581E090E00E947E04C090BE
:103E10002301D0902401E0902501F09026012DECA3
:103E20003CEC4CE450E4C501B4010E940E2787FD30
:103E300020C02DEC3CEC4CE450E46091A505709161
:103E4000A6058091A7059091A8050E940E2787FDE1
:103E500010C02DEC3CEC4CE450E46091A105709155
:103E6000A2058091A3059091A4050E940E2787FFCB
:103E700031C080915705882321F085EF91E00E94A1
:103E8000860E8091680590916905A0916A05B091B0
:103E90006B0540910C0550910D0560910E057091D8
:103EA0000F05841B950BA60BB70B81309D4DAD46BE
:103EB000B10528F08DE290E00E94240622C285E040
:103EC00090E00E9424067AE9C72E79E9D72EED2CDE
:103ED0007EE3F72E29E23CE54FE05EE3C701B60141
:103EE0000E94A1269B01AC016091950570919605F9
:103EF00080919705909198050E946D2887FD3CC0A0
:103F00002AE037ED43EA5CE360918B0570918C0504
:103F100080918D0590918E050E94A22620913901F5
:103F200030913A0140913B0150913C010E940E2793
:103F3000181614F1A70196016091140170911501F2
:103F400080911601909117010E940E27811104C0E3
:103F500080916105811102C00E945709C09214012D
:103F6000D0921501E0921601F092170181E0809342
:103F700061051092620531C02AE037ED43E25CE34F
:103F80006091390170913A0180913B0190913C011F
:103F90000E94A1266B017C019B01AC016091100184
:103FA0007091110180911201909113010E940E27CE
:103FB000811104C080916205811102C00E945709DD
:103FC000C0921001D0921101E0921201F0921301FF
:103FD00081E0809362051092610580914405811112
:103FE00090C18091680590916905A0916A05B09192
:103FF0006B0540910C0150910D0160910E01709183
:104000000F018C019D01041B150B260B370B4091F2
:104010008705509188056091890570918A05401740
:1040200051076207730708F06CC18093870590936E
:104030008805A0938905B0938A0584EC99E0A0E0F7
:10404000B0E080930C0190930D01A0930E01B0930A
:104050000F0120906705909166059D83A0916505ED
:10406000A987C090A905D090AA05E090AB05F09073
:10407000AC054090A5055090A6056090A7057090EE
:10408000A8058090A1059090A205A090A305B090EE
:10409000A405A3019201C701B6010E94A1262DEC3F
:1040A0003CEC4CE45DE30E946D281816FCF0A50181
:1040B0009401C701B6010E94A1262DEC3CEC4CE412
:1040C0005DE30E946D281816A4F4332433942091E4
:1040D0002701309128014091290150912A01C701FF
:1040E000B6010E946D2818162CF003C033243394B7
:1040F00001C0312CA7019601C301B2010E94A12683
:104100002DEC3CEC4CE45DE30E946D281816F4F0B5
:10411000A5019401C301B2010E94A1262DEC3CEC43
:104120004CE45DE30E946D28181694F401E02091A0
:104130002701309128014091290150912A01C301A2
:10414000B2010E946D28181624F002C001E001C0DF
:1041500000E0A7019601C501B4010E94A1262DEC43
:104160003CEC4CE45DE30E946D281816F4F0A301CA
:104170009201C501B4010E94A1262DEC3CEC4CE457
:104180005DE30E946D28181694F411E02091270138
:10419000309128014091290150912A01C501B401B3
:1041A0000E946D28181624F002C011E001C010E032
:1041B0003320C1F0A3019201C701B6010E940E276E
:1041C00087FF08C0A5019401C701B6010E940E2710
:1041D00087FD08C061E088E00E942C0381E08093A5
:1041E000670506C060E088E00E942C031092670516
:1041F000002361F1C090A505D090A605E090A70529
:10420000F090A8052091A9053091AA054091AB0531
:104210005091AC05C701B6010E940E2787FF0EC062
:104220002091A1053091A2054091A3055091A405CC
:10423000C701B6010E940E2787FD08C060E087E035
:104240000E942C0381E08093660506C061E087E050
:104250000E942C0310926605112361F1C090A10504
:10426000D090A205E090A305F090A4052091A905A7
:104270003091AA054091AB055091AC05C701B6013C
:104280000E940E2787FF0EC02091A5053091A6053C
:104290004091A7055091A805C701B6010E940E27BD
:1042A00087FD08C060E084E00E942C0381E08093D9
:1042B000650506C061E084E00E942C03109265054C
:1042C000311004C0011102C0112361F020E23EE46C
:1042D00040E050E020930C0130930D0140930E011B
:1042E00050930F0180916705821109C08091660586
:1042F0003D81831304C080916505498584130E9424
:1043000057098091680590916905A0916A05B0915F
:104310006B058C019D010858134121093109409119
:10432000C7055091C8056091C9057091CA0540172D
:1043300051076207730708F0C1C1883853E1950738
:10434000A105B10508F4BAC1409131015091320183
:104350006091330170913401483C5105610571054C
:1043600009F4ACC1209157052111A8C18093C7055C
:104370009093C805A093C905B093CA0587E092E061
:104380000E942D1080912001909121018130910592
:1043900019F48BE092E009C0009719F489E092E0EB
:1043A00004C0019621F483E192E00E942D10209137
:1043B0001C0130911D0140911E0150911F0160911F
:1043C0004B0570914C0580914D0590914E050E94D2
:1043D000132720E030E048EC52E40E9472280E944B
:1043E0008527072E000C880B990B0E9403108CE187
:1043F00092E00E942D108091D505882321F08EE156
:1044000092E00E942D1088E292E00E942D1080918F
:10441000D505882309F498C06091B5057091B6055B
:104420008091B7059091B8050E942F1080E392E02B
:104430000E942D106091B1057091B2058091B30575
:104440009091B4050E942F1080E392E00E942D10FD
:104450006091AD057091AE058091AF059091B0056A
:104460000E942F1082E392E00E942D106091A90516
:104470007091AA058091AB059091AC050E942F1018
:1044800080E392E00E942D106091A5057091A60531
:104490008091A7059091A8050E942F1080E392E0DB
:1044A0000E942D106091A1057091A2058091A30535
:1044B0009091A4050E942F1089E392E00E942D1094
:1044C00080916705882319F082E694E002C08CE9A8
:1044D00093E00E942D1080916605882319F082E6F2
:1044E00094E002C08CE993E00E942D108091650554
:1044F000882319F082E694E002C08CE993E00E94E0
:104500002D1080914405882321F08EE392E00E94D3
:104510002D1080E492E00E942D1060919D05709115
:104520009E0580919F059091A0050E942F1086E422
:1045300092E00E942D106091990570919A058091EA
:104540009B0590919C0532C06091240570912505D2
:1045500080912605909127050E942F1080E392E01C
:104560000E942D10609120057091210580912205F7
:10457000909123050E942F1080E392E00E942D105D
:1045800060911C0570911D0580911E0590911F057D
:104590000E942F108CE492E00E942D10609118056B
:1045A0007091190580911A0590911B050E942F109A
:1045B00081E592E00E942D10609163057091640581
:1045C000072E000C880B990B0E94031087E592E0E0
:1045D0000E942D108091D505882349F060919505A2
:1045E00070919605809197059091980508C060910B
:1045F00014057091150580911605909117050E947C
:104600002F108EE592E00E942D1060914B05709165
:104610004C0580914D0590914E050E948527072EEF
:10462000000C880B990B0E94031084E692E00E9414
:104630002D10609118017091190180911A019091CB
:104640001B010E942F1020E030E046EC52E4209342
:1046500018013093190140931A0150931B0189E608
:1046600092E00E942D1060911005709111058091CB
:104670001205909113050E942F108EE692E00E9481
:104680002D1080912201882319F08CE993E002C05B
:1046900082E694E00E942D1083E792E00E942D10A4
:1046A0006091280570912905072E000C880B990B45
:1046B0000E94031088EC92E00E94860E80916805AB
:1046C00090916905A0916A05B0916B058C019D01DF
:1046D000005E13492440310940914F055091500527
:1046E0006091510570915205401751076207730799
:1046F000F8F4803E33E9930734E0A307B105C0F036
:1047000080934F0590935005A0935105B0935205A7
:1047100060914B0570914C0580914D0590914E052F
:104720000E948527DC01CB0160E070E00E940B064F
:104730008091470590914805A0914905B0914A059F
:10474000409168055091690560916A0570916B050B
:1047500084179507A607B70730F4892B8A2B8B2B74
:1047600011F00E948B0780914505909146050E94AB
:104770007E048091680590916905A0916A05B091C9
:104780006B058C019D0100581F4422413109409165
:10479000C3055091C4056091C5057091C6054017C9
:1047A000510762077307C8F480384FE4940742E169
:1047B000A407B10590F08093C3059093C405A0931E
:1047C000C505B093C60587E090E00E94240681E00D
:1047D00090E09093300180932F0180916805909133
:1047E0006905A0916A05B0916B054091D60550917D
:1047F000D7056091D8057091D905841B950BA60B40
:10480000B70B813C944DA140B10540F08091440527
:10481000882321F08CE290E00E94240680916805B4
:1048200090916905A0916A05B0916B058C019D017D
:104830000A50110921093109409140055091410563
:104840006091420570914305401751076207730755
:1048500008F09EC08A309105A105B10508F498C002
:104860008093400590934105A0934205B093430582
:104870008EE00E94DB032091C1053091C205820FBA
:10488000931F9093C2058093C1058FE00E94DB03C4
:104890002091BF053091C005820F931F9093C005F2
:1048A0008093BF0580E10E94DB032091BD0530911C
:1048B000BE05820F931F9093BE058093BD0581E1D5
:1048C0000E94DB037C018091BB059091BC058E0D9D
:1048D0009F1D9093BC058093BB0582E10E94DB0382
:1048E0008C018091B9059091BA05800F911F90932A
:1048F000BA058093B9058091D3059091D4050196AE
:104900009093D4058093D305B701FF0C880B990BC6
:104910000E94BD2720E030EC4FE754E40E941327AB
:104920002FE632E143E850E40E9472286B017C01DB
:10493000B801110F880B990B0E94BD2720E030ECC5
:104940004FE754E40E9413272FE632E143E850E496
:104950000E94722827E53FE348E65EE30E941327A2
:104960004B015C012FEF35EE42E95EE3C701B60172
:104970000E9413279B01AC01C501B4010E946D2860
:10498000181634F480912201811102C00E94920510
:1049900088EE95E00E940302181619060CF09EC0DE
:1049A0008091310190913201A0913301B091340195
:1049B000883C9105A105B10509F490C088EE95E009
:1049C0000E94E10140913A0550913B059A012F5F09
:1049D0003F4F30933B0520933A05FA01EE0FFF1F3E
:1049E000E65DFA4F918380838D30910509F4EFC025
:1049F0008A30910509F4EBC040912A0550912B05AE
:104A00004533510509F4FCC04434510509F4F8C09C
:104A10004834510509F4F4C08D30910509F4F7C00C
:104A20000A9709F4F4C08091680590916905A091F6
:104A30006A05B0916B058093C3059093C405A0935C
:104A4000C505B093C6058091280590912905079763
:104A500009F040C080E090E00E9424068DEC9CECC0
:104A6000A4E8B0E48093390190933A01A0933B010C
:104A7000B0933C0123E333E343E850E420938906F9
:104A800030938A0640938B0650938C0683E393E31E
:104A9000A3E7B0E480932B0190932C01A0932D0108
:104AA000B0932E018DEC9CECACE4B0E48093270134
:104AB00090932801A0932901B0932A0120E030E0CF
:104AC00040E85FE3209323013093240140932501C4
:104AD000509326011092300110922F0180913C05D5
:104AE00090913D05A0913E05B0913F050097A1052D
:104AF000B10509F468C0409168055091690560915D
:104B00006A0570916B05481759076A077B0708F417
:104B10005AC060914B0570914C0580914D05909164
:104B20004E050E948527DC01CB0160E070E00E9409
:104B30000B0661E08DE00E942C0360E07DE780E0E1
:104B400090E00E94F80360E08DE00E942C0360E09A
:104B50007DE780E090E00E94F80361E08DE00E9434
:104B60002C0360E07DE780E090E00E94F80360E0C5
:104B70008DE00E942C0360E07DE780E090E00E94E1
:104B8000F80361E08DE00E942C0360E07DE780E0A7
:104B900090E00E94F80360E08DE00E942C0360E04A
:104BA0007DE780E090E00E94F8030E946E0788E7AE
:104BB00092E00E94860E10923C0510923D051092E4
:104BC0003E0510923F050E94A3020C942E126091A4
:104BD0002A0570912B056533710509F40DCF6434F6
:104BE000710509F409CF6834710509F405CF12166F
:104BF00013060CF001CF50933B0540933A0504C0D7
:104C00002330310509F008CF0E948E0904C02130FD
:104C1000310509F008CF10923B0510923A0503CFF9
:104C2000E8EEF5E01382128288EE93E0A0E0B0E0B7
:104C300084839583A683B78381E491E09183808305
:104C400085EC90E09587848784EC90E09787868751
:104C500080EC90E0918B808B81EC90E0938B828B49
:104C600082EC90E0958B848B86EC90E0978B868B22
:104C7000118E128E138E148E2DEC3CEC4CE45DE301
:104C80006091390170913A0180913B0190913C0112
:104C90000E94A1266093890670938A0680938B06F2
:104CA00090938C062AE939E949E15FE36091350187
:104CB0007091360180913701909138010E94A126B0
:104CC0006093850670938606809387069093880686
:104CD0000895F999FECF92BD81BDF89A992780B5C4
:104CE0000895262FF999FECF1FBA92BD81BD20BD30
:104CF0000FB6F894FA9AF99A0FBE01960895A1E2B8
:104D00001A2EAA1BBB1BFD010DC0AA1FBB1FEE1F45
:104D1000FF1FA217B307E407F50720F0A21BB30B90
:104D2000E40BF50B661F771F881F991F1A9469F70C
:104D300060957095809590959B01AC01BD01CF0168
:104D400008955058BB27AA270E94B9260C943328EF
:104D50000E94252838F00E942C2820F039F49F3F2B
:104D600019F426F40C9422280EF4E095E7FB0C9439
:104D70001C28E92F0E94442858F3BA1762077307CA
:104D80008407950720F079F4A6F50C9466280EF4B4
:104D9000E0950B2EBA2FA02D0B01B90190010C014B
:104DA000CA01A0011124FF27591B99F0593F50F463
:104DB000503E68F11A16F040A22F232F342F4427BB
:104DC000585FF3CF469537952795A795F0405395B3
:104DD000C9F77EF41F16BA0B620B730B840BBAF083
:104DE0009150A1F0FF0FBB1F661F771F881FC2F7EE
:104DF0000EC0BA0F621F731F841F48F48795779502
:104E00006795B795F7959E3F08F0B0CF9395880FBB
:104E100008F09927EE0F9795879508950E94F82737
:104E200008F481E008950E9427270C9433280E94FB
:104E30002C2858F00E94252840F029F45F3F29F0E3
:104E40000C941C2851110C9467280C9422280E9461
:104E5000442868F39923B1F3552391F3951B550B1F
:104E6000BB27AA2762177307840738F09F5F5F4F3D
:104E7000220F331F441FAA1FA9F335D00E2E3AF07C
:104E8000E0E832D091505040E695001CCAF72BD094
:104E9000FE2F29D0660F771F881FBB1F26173707E5
:104EA0004807AB07B0E809F0BB0B802DBF01FF2717
:104EB00093585F4F3AF09E3F510578F00C941C28B0
:104EC0000C9467285F3FE4F3983ED4F3869577957A
:104ED0006795B795F7959F5FC9F7880F911D9695D0
:104EE000879597F90895E1E0660F771F881FBB1F2C
:104EF000621773078407BA0720F0621B730B840BD9
:104F0000BA0BEE1F88F7E09508950E948C276894ED
:104F1000B1110C94672808950E944C2888F09F577F
:104F200098F0B92F9927B751B0F0E1F0660F771FCD
:104F3000881F991F1AF0BA95C9F714C0B13091F0C3
:104F40000E946628B1E008950C946628672F782F98
:104F50008827B85F39F0B93FCCF386957795679588
:104F6000B395D9F73EF490958095709561957F4FF4
:104F70008F4F9F4F0895E89409C097FB3EF490959A
:104F80008095709561957F4F8F4F9F4F9923A9F022
:104F9000F92F96E9BB279395F695879577956795B1
:104FA000B795F111F8CFFAF4BB0F11F460FF1BC0F5
:104FB0006F5F7F4F8F4F9F4F16C0882311F096E988
:104FC00011C0772321F09EE8872F762F05C0662336
:104FD00071F096E8862F70E060E02AF09A95660FEF
:104FE000771F881FDAF7880F9695879597F90895A8
:104FF000990F0008550FAA0BE0E8FEEF16161706EA
:10500000E807F907C0F012161306E407F50798F051
:10501000621B730B840B950B39F40A2661F0232B6A
:10502000242B252B21F408950A2609F4A140A695E6
:105030008FEF811D811D089597F99F6780E870E0CB
:1050400060E008959FEF80EC089500240A941616FE
:10505000170618060906089500240A941216130666
:10506000140605060895092E0394000C11F48823F4
:1050700052F0BB0F40F4BF2B11F460FF04C06F5F10
:105080007F4F8F4F9F4F089557FD9058440F551FE6
:1050900059F05F3F71F04795880F97FB991F61F0BA
:1050A0009F3F79F087950895121613061406551F31
:1050B000F2CF4695F1DF08C0161617061806991F9D
:1050C000F1CF86957105610508940895E894BB2792
:1050D00066277727CB0197F908950E94F82708F4EF
:1050E0008FEF08950E9485280C9433280E9425286C
:1050F00038F00E942C2820F0952311F00C941C28E5
:105100000C94222811240C9467280E94442870F3E0
:10511000959FC1F3950F50E0551F629FF001729F5C
:10512000BB27F00DB11D639FAA27F00DB11DAA1F6B
:10513000649F6627B00DA11D661F829F2227B00DB8
:10514000A11D621F739FB00DA11D621F839FA00D43
:10515000611D221F749F3327A00D611D231F849F93
:10516000600D211D822F762F6A2F11249F575040EA
:105170009AF0F1F088234AF0EE0FFF1FBB1F661F65
:10518000771F881F91505040A9F79E3F510580F02E
:105190000C941C280C9467285F3FE4F3983ED4F3EA
:1051A000869577956795B795F795E7959F5FC1F7D2
:1051B000FE2B880F911D9695879597F908950E946B
:1051C000F827880B990B089597FB072E16F4009487
:1051D00007D077FD09D00E94F82807FC05D03EF4DF
:1051E000909581959F4F0895709561957F4F089593
:1051F000AA1BBB1B51E107C0AA1FBB1FA617B707FD
:1052000010F0A61BB70B881F991F5A95A9F7809518
:105210009095BC01CD010895EE0FFF1F0590F4910C
:10522000E02D099481E090E0F8940C941729F8940B
:02523000FFCFAE
:10523200011400FFFF01000088C00500C40900003E
:10524200333383400000003F0000C64200D0844553
:10525200FFFF010000803FCDCC4C4033337340FF51
:10526200FFD007000000006041CDCC844000000068
:10527200003A02A301D20181020302E101F5013CDD
:1052820072657365743E00686967682043484152DD
:1052920047494E472063656C6C0068696768206304
:1052A200757272656E74003C646F636B65643E0078
:1052B2006175746F20636861726765204F4E003CB0
:1052C200756E646F636B65643E006175746F206315
:1052D2006861726765204F4646003C77616C6C706E
:1052E2006F7765723E0064616E6765726F75736C8D
:1052F20079206C6F772063656C6C003C7265646F1B
:10530200636B3E003C686967685F63757272656EC5
:10531200743E000A6D61782063686172676520746B
:10532200696D650A000A707265636F6E64697469FB
:105332006F6E696E670A003C00756E646F636B6521
:10534200642000756E6B6E6F776E200025005F63C0
:1053520068617267696E67002063656C6C733A00FE
:105362005F005F69646C653A005F73683A004100F0
:105372005F7343563A005F7349563A005F73563A79
:10538200005F70776D3A005F616D70733A005F6D18
:1053920041683A005F6C563A005F63433A005F62CD
:1053A200503A005F65523A003C5348555454494EB6
:1053B20047444F574E3E0062617474506C7573508F
:1053C200696E20484947482028666C6F7729006239
:1053D200617474506C757350696E204C4F5720285D
:1053E2006E6F20666C6F7729003C706F7765725F15
:1053F2006572726F722000303E002C007772697401
:10540200696E67206572726F7220746F20656570B5
:10541200726F6D003C72656D6F76655F77616C6C63
:10542200706F7765723E00626174742073616665A5
:10543200747920737769746368204F4646000A7A4C
:1054420065726F2063757272656E740A006E65779D
:105452002063757272656E742063616C3A20003C41
:1054620073687574646F776E3E003C63686172673F
:1054720065643E007368756E7431204F4646007352
:1054820068756E7431204F4E007368756E743220E9
:105492004F4646007368756E7432204F4E00736833
:1054A200756E7433204F4646007368756E743320F0
:1054B2004F4E007368756E747320616C6C206F665A
:1054C2006600766F6C74732050574D203000766FF3
:1054D2006C74732050574D2031303000766F6C74ED
:1054E200732050574D2032303000766F6C74732029
:1054F20050574D203235350061646A566F6C7473B3
:10550200204F46460061646A566F6C7473204F4E9A
:105512000061646A416D7073204F46460061646A9F
:10552200416D7073204F4E00746172676574204143
:105532006D7073202B302E30350074617267657484
:1055420020416D7073202D302E30350074617267EA
:10555200657420766F6C7473202B302E3032007499
:10556200617267657420766F6C7473202D302E30F3
:10557200323A200070777250574D202B3130007034
:10558200777250574D202D31300070777250574D41
:10559200202B310070777250574D202D31006675E7
:1055A2006C6C6175746F204F46460066756C6C6159
:1055B20075746F204F4E003C69643A3A6F63756CA4
:1055C2007573506F7765723E006261747420736107
:1055D2006665747920737769746368204F4E003C66
:1055E2006D416843617061636974793A20003C6D72
:1055F20041683A20003C656570726F6D5F6572614B
:105602007365643E003C77726974696E675F746F9C
:105612005F656570726F6D3E003C646F636B566FC1
:105622006C746167653A20000D0A006E616E006954
:085632006E66006F7666000051
:00000001FF
